:020000040002F8
:10600000B04C0020F9620200016302000363020049
:10601000056302000763020009630200000000003C
:106020000000000000000000000000000B63020000
:106030000D630200000000000F6302001163020004
:1060400089650200136302002969020013630200DC
:106050001363020013630200C163020013630200B2
:106060001363020013630200136302001363020050
:106070001363020013630200136302001363020040
:1060800013630200E1650200136302001363020060
:106090000566020013630200096602001363020032
:1060A0001363020013630200136302001363020010
:1060B00013630200136302000000000000000000F0
:1060C00013630200136302001363020013630200F0
:1060D0001363020013630200136302000000000058
:1060E00000000000000000000000000000000000B0
:1060F00000000000000000000000000000000000A0
:10610000000000000000000000000000000000008F
:10611000000000000000000000000000000000007F
:10612000000000000000000000000000000000006F
:10613000000000000000000000000000000000005F
:10614000000000000000000000000000000000004F
:10615000000000000000000000000000000000003F
:10616000000000000000000000000000000000002F
:10617000000000000000000000000000000000001F
:10618000000000000000000000000000000000000F
:1061900000000000000000000000000000000000FF
:1061A00000000000000000000000000000000000EF
:1061B00000000000000000000000000000000000DF
:1061C00000000000000000000000000000000000CF
:1061D00000000000000000000000000000000000BF
:1061E00000000000000000000000000000000000AF
:1061F000000000000000000000000000000000009F
:10620000DFF80CD000F0CAF800480047898002008F
:10621000B04C002030B4044654E8000F0D4644E86A
:106220000053002BF8D1156030BC704730B40446E1
:1062300054E8000F40EA010544E80053002BF7D171
:10624000156030BC704730B4044654E8000F00EAD3
:10625000010544E80053002BF7D1156030BC7047AE
:1062600030B4044654E8000F80EA010544E80053C6
:10627000002BF7D1156030BC704730B4044654E8A9
:10628000000F00EB010544E80053002BF7D1156027
:1062900030BC704730B4044654E8000FA0EB010551
:1062A00044E80053002BF7D1156030BC704770B440
:1062B00004464FF0000054E8006F0D68AE4207BF7F
:1062C00044E80023012044E800630E60002B1CBF5B
:1062D0000020F0E770BC704730B4044654E8000F6B
:1062E00088422CBF451A054644E80053002BF5D1DF
:1062F000156030BC704700000648804706480047DC
:10630000FEE7FEE7FEE7FEE7FEE7FEE7FEE7FEE765
:10631000FEE7FEE70D66020001620200202A04DBB0
:10632000203A00FA02F1002070479140C2F12003A8
:1063300020FA03F31943904070470000004870476B
:1063400068AF020040EA01039B0703D009E008C9D7
:10635000121F08C0042AFAD203E011F8013B00F82A
:10636000013B521EF9D27047D2B201E000F8012B76
:10637000491EFBD270470022F6E710B513460A46C5
:1063800004461946FFF7F0FF204610BD421C10F8E6
:10639000011B0029FBD1801A70470000064C074DF5
:1063A00006E0E06840F0010394E8070098471034E5
:1063B000AC42F6D3FFF728FF6CB602008CB60200A1
:1063C0002DE9F04700268AB0DFF85091B0464FF42F
:1063D0008075012437460696284602F011FC38B134
:1063E000D9F80403204203D0284602F0FFFB2643DD
:1063F0002D1D64007F1CADB2082FEDD34FF4BE7489
:10640000204602F0FDFB48B1204602F0EFFB46F0CB
:10641000004606AA0121002002F0D4FB404D16F0F0
:10642000FF0F15D00127002437420DD009EB84015E
:10643000D1F81005D1F81015C0F3042055F8242028
:10644000C1F3014102B190477F00641C082CEBD3DB
:10645000002E5FDA4FF0FF30CDF8108054E028199D
:1064600010F8507F90F9000027F0C008401C3BD086
:1064700007A9404602F049F810B34FEA9719404681
:1064800001F03AF955F820701FB1B9F1030F03D0AC
:1064900006E0B9F1030F27D104A9404602F03DF808
:1064A0004FF0A04101EB8800D0F8000706A9C0F327
:1064B000014A404602F029F818B1BAF1020F03D0A0
:1064C00012E0BAF1030F0FD1B9F1030F08D1BAF1FD
:1064D000020F1DD00221404602F058FB761CF6B296
:1064E00017B149464046B847641C042CB7D3002E68
:1064F00010D06A460121002002F064FB0699009842
:10650000884207D006900498002634460790A6E7F4
:106510000321E0E70AB0BDE8F0870000006000401A
:106520000025002000F01F02012191404009800059
:1065300000F1E020C0F88012704700F01F02012136
:1065400091404009800000F1E020C0F80011704740
:1065500000F01F02012191404009800000F1E0207D
:10656000C0F8001270474907090E002806DA00F04B
:106570000F0000F1E02080F8141D704700F1E020CA
:1065800080F800147047000070B54FF480763046F4
:1065900002F0FEF8114CB50560B1304602F0FFF88C
:1065A0000120C5F80803607920B9012060712168D5
:1065B000002088474FF48276304602F0E9F8002840
:1065C0000AD0304602F0EBF80220C5F80803216833
:1065D000BDE870400120084770BD0000E82200209F
:1065E00007480021C0F84011C0F84411C0F8481114
:1065F000C0F84C11C0F80011C0F8041104F03AB80A
:106600000010014003F084BF03F04CB8F0B5B5486A
:106610000023021D0178101D01254FF0805406292A
:106620000BD11678360708D10678C6F30316032E69
:1066300006D0042E04D0052E02D0062907D00EE085
:10664000B4F82463A84FC6F304263E6002E016782F
:10665000360704D10678C6F30316032E02D00629A6
:1066600004D00FE0A24FA14E7E670EE016783607E9
:1066700008D10678C6F30316032E06D0042E04D0E4
:10668000052E02D0062907D00EE0D4F84462994FB7
:10669000C6F342363E6002E01678360704D106782B
:1066A000C6F30316032E02D0062906D011E0924E3F
:1066B000376827F0807737600EE01678360708D104
:1066C0000678C6F30316032E06D0042E04D0052E3A
:1066D00002D006290AD011E04FF08046C6F80C31EE
:1066E000C6F81031834E361F336002E01678360745
:1066F00004D10678C6F30316032E02D0062905D06E
:106700000CE07C4F032664373E600AE016783607BB
:1067100004D10678C6F30316032E02D006290DD045
:1067200014E0764F05263E60744E78363560734E21
:10673000083633603F263F1D3E6002E0167836077C
:1067400004D10678C6F30316052E02D0062957D0C9
:1067500062E06B4E36686B4F3E60694E361D3668A0
:106760003F1D3E60664E083636683F1D3E60644EF3
:106770000C3636683F1D3E60614E103636683F1D50
:106780003E605F4E143636683F1D3E605C4E1836E4
:1067900036685C4F20373E60594E1C3636683F1DC8
:1067A0003E60574E203636683F1D3E60544E2436BC
:1067B00036683F1D3E60524E283636683F1D3E60AB
:1067C0004F4E2C3636683F1D3E604D4E3036366893
:1067D0004C4F40373E604A4E343636683F1D3E606F
:1067E000474E383636683F1D3E60454E3C3636686B
:1067F0003F1D3E60424E403636683F1D3E6002E01F
:106800001678360708D10678C6F30316032E06D08D
:10681000042E04D0052E02D0062907D019E0D4F8A2
:106820005812394A01F04F01116002E0117809074E
:106830000FD10078C0F30310032803D0042801D03F
:10684000052806D131480168C90702D06FF001015F
:106850000160D4F83001062808D1D4F834010628A4
:1068600004D12B48016841F48061016022487438EA
:10687000016841F470010160BFF34F8FBFF36F8F68
:106880004FF01021D1F80002002803DBD1F80402F8
:10689000002822DA1F4A15601F480468002CFCD02B
:1068A0001524C1F800420568002DFCD0C1F804424F
:1068B00001680029FCD0136001680029FCD0BFF3F7
:1068C0004F8F0D48F0380168144A01F4E06111431C
:1068D0000160BFF34F8F00BFFDE712491048086009
:1068E000F0BD0000E00F00F0403501400DF0ADBA02
:1068F00000C007403C050040FCED00E010560040A1
:106900000404001020C50040E40E004000040040D4
:106910003C17004004E5014000E401400400FA0592
:106920000090D003A8230020014800680047000021
:10693000F022002002E008C8121F08C1002AFAD184
:1069400070477047002001E001C1121F002AFBD1EF
:10695000704700000121202803DA814005480140EA
:1069600003E0402802DA2038814009B10120704755
:1069700000207047FC06FFBD30B52548A5B03C217E
:10698000006824902348807C8DF892006846FFF7C9
:10699000F2FC02208DF8000001248DF80240062050
:1069A0008DF803003C210FA8FFF7E5FC24A81A4D41
:1069B0001490ADF84C402A1D6846296800F048FA4A
:1069C00008B100F0E3F8144A0FA80C32A96800F0EF
:1069D0003FFA08B100F0DAF818211EA8FFF7CBFC47
:1069E00000208DF88D408DF87840ADF884001F9020
:1069F0008DF88C004020084920901EAAA1F10C00BF
:106A000072DF002801D000F0C1F825B030BD0000D1
:106A100044AC0200AC230020C4220020064810B57C
:106A20000121007873DF08B100F0B0F8BDE8104034
:106A3000002000F077BD0000B822002070B50024CF
:106A4000084D05E0686810F8340002F007FF641C88
:106A500028788442F6D304484068BDE8704000F0CE
:106A600021B90000F822002084AC020070B5002497
:106A7000064D06E06868012110F8340002F012FFAC
:106A8000641C28788442F5D3002070BDF8220020D1
:106A9000F8B515460C460646052A01D20720F8BD72
:106AA00002F0FAFF18B902F0C1FF0028F7D112492D
:106AB00000224E600C708D60C1E90422C1E90622FB
:106AC0000E4D0DE006EBC4002968009181788DF829
:106AD000011000780A4A694602F036FF0028DED12C
:106AE000641EE4B2EED2BDE8F84004480021054A35
:106AF000001D00F057B80000F822002084AC02000E
:106B00004D7C02005D7B020072B602F01BFB00BFF1
:106B100002F05CF90028FBD111481249401AC40860
:106B2000012000EB044010A102F06AFA114800684D
:106B3000C00700D000BE022000EB04400EA102F00E
:106B40005FFABFF34F8F0B48E43801680E4A01F437
:106B5000E06111430160BFF34F8F00BFFDE700000C
:106B6000DCB602009CB60200466174616C2065725E
:106B7000726F7200F0ED00E053797374656D2072EE
:106B800065736574000000000400FA050EB500216D
:106B90000091CDE901106A4644F20100FFF7B4FF0D
:106BA0000EBD0000074B9B7823B12AB120B10068CD
:106BB000037C1BB108207047072070474174426175
:106BC00000207047CC25002070B503F0FBFA104878
:106BD00000240B21047044700E4D817014206C60F1
:106BE0002C706C70FFF79EFC06211420FFF7BBFC95
:106BF0001420FFF7A2FC0848046006211120FFF7CB
:106C0000B2FC0548001F0068A860002070BD0000AD
:106C1000CC25002018230020081501402DE9FC4751
:106C2000DFF8789099F8023073B368B3052902D27F
:106C30000720BDE8FC87436933B3437C012B25D093
:106C4000002704460025884616468DF80050684601
:106C500000F038F801A803F075FFC8B101210170F8
:106C60000F4944600968C0E90218C0E904769DF83C
:106C7000040089F801009DF8000000F047F8142096
:106C8000FFF766FC2846D4E70820D2E70F46D8E78E
:106C900004259DF8000000F039F8F3E7CC2500202A
:106CA000041501400649897839B130B1416921B1F3
:106CB00000210174022103F0B9BC082070470000D4
:106CC000CC25002030B5EFF3108172B60D4A9468E0
:106CD000012324B10370002900D162B630BD936056
:106CE0004FF0E023D3F88051074C25401560C3F8DE
:106CF0008041D3F8844154605A17C3F8842100229C
:106D00000270E8E7D8260020FC06FFBD0B498A6820
:106D1000002A11D000280FD1EFF3108072B60B6853
:106D20004FF0E022C2F800314B68C2F80431002273
:106D30008A60002800D162B670470000D826002083
:106D40002DE9F041064608680C46411C4FF0A0476B
:106D50004FF0010506D005FA00F1C7F808152068C4
:106D600001F000FF6068411C02D0002101F0E8FE44
:106D70003168A069C1F82405607D227D3168104327
:106D8000C1F86C05D4E900123068C0F81425C0F8C9
:106D90000C15207D012815D1A068411C02D00021CE
:106DA00001F0CEFEE068411C05D08540C7F80855CB
:106DB000E06801F0D7FED4E902123068C0F8082577
:106DC000C0F81015BDE8F0812DE9F04106460868CD
:106DD0000C46411C4FF0A0474FF0010506D005FAC4
:106DE00000F1C7F80815206801F0C6FE6068411C74
:106DF00002D0002101F0ADFE3168A069C1F8240580
:106E0000607D217D32680843C2F86C05D4E9001228
:106E10003068C0F80C15C0F81425207D012815D164
:106E2000A068411C02D0002101F093FEE068411CE3
:106E300005D08540C7F80855E06801F09DFED4E90B
:106E400002123068C0F80825C0F81015BDE8F081BE
:106E50002DE9FC47002517880646158090F82D007F
:106E60001446894630B13A462146484600F0E6F8D5
:106E7000051E09D1B0784FF00C0A18B32088C84617
:106E8000001DB84202D95046BDE8FC87684679DF4C
:106E90000028F9D12088032108F800102088192142
:106EA000401C80B2208008F800102088401C80B26E
:106EB000208000EB0801BDF8000003F09EFD218852
:106EC00008442080F0780222C8B1218896F9033066
:106ED00001F1030C4846BC45D5D8425421884FF0F7
:106EE000010C491C89B2218000F801C02188491C8D
:106EF00089B2218009F801302088401C2080706808
:106F0000B8B1218890F9003001F1030C4846BC4526
:106F1000B9D8425421880A22491C89B2218042549E
:106F20002188491C89B2218009F801302088401C41
:106F30002080308950B1CDE900474B46062202211E
:106F400006F1080003F016FE051E9DD1308A50B1EF
:106F5000CDE900474B460722032106F1100003F05C
:106F600009FE051E90D1308B50B1CDE900474B464C
:106F70001522142106F1180003F0FCFD051E83D133
:106F8000306A30B13B462246494600F01CFD051EE2
:106F9000DBD1706A30B13B462246494601F03EF9EA
:106FA000051ED2D196F82C0038B13B462246494600
:106FB000304603F0D3F9051EC7D1307838B13B46CF
:106FC00022464946304601F0B3F9051EBDD1284698
:106FD0005AE7000070B5040012D001461C22144884
:106FE000FFF7B0F91248134D0560206850B17ADF01
:106FF000002806D12068016829604068686005E0C3
:107000000E2070BD0B487BDF0028FAD108484FF6F0
:10701000FF711438084A20F8041B0549343901600F
:107020000021FFF7BFFD0028EBD0032070BD00005A
:1070300058240020D4220020B9AA02007CB50546BD
:1070400008880C460930904201D90C207CBD684666
:107050006DDF0028FAD121880820685420881B2180
:10706000401C80B2208029542088401C80B220809F
:107070002844DDF801100160BDF8051081802088EA
:10708000801D80B220809DF80010490800D00121A9
:1070900029542088401C208000207CBDF8B5334D49
:1070A000018804466E8821294BD015DC3048314ACE
:1070B0001029A0EB02004FEAD0004FF0030202EBD0
:1070C000004013D011292AD0132943D100231A4696
:1070D000852130467FDF1CE03B2942D052293AD03F
:1070E000562937D18088132176DF12E022A101F0E2
:1070F00087FF012000F016FA002000F00BFAA188AB
:107100006980204801F0CCFA08B1FFF73FFDFFF796
:10711000ADFC00281ED0BDE8F840FFF737BD1AA12E
:1071200001F06EFF012000F0F5F94FF6FF70688066
:10713000FFF784FC08B1FFF729FDBDE8F840FFF731
:107140006DBC00200090A08869468FDF002801D028
:10715000FFF71CFDF8BD00231A4619463046B1DF83
:10716000D7E78088132176DFD3E70000B82200201C
:10717000DCB602009CB60200436F6E6E65637465F8
:1071800064000000D8230020446973636F6E6E654D
:1071900063746564000000002DE9F04701883B4EF0
:1071A00040F2F3194FF6FF7510291BD011293ED07C
:1071B000122954D0502946D1C188F289841D9142A8
:1071C00041D1618902293ED18688304600F080FD98
:1071D000050038D004F10C0000F06EF9A8B3294680
:1071E00030464EE0C17B8788044601292BD1A84652
:1071F000284600F06DFD050017D02F800020287272
:10720000234843464A460168C5F80A104068C5F855
:107210000E0004F1100105F10A0000F00FFE687283
:10722000F08900280FD129462AE0042013E0808845
:1072300000F04EFD040006D06068FFF733FD08B192
:1072400003F064F82580BDE8F087FFE76868FFF782
:1072500029FD0028F7D0BDE8F04703F057B887882C
:107260000646384600F034FD0400ECD02B464A4672
:1072700006F1080104F10A0000F0E0FD6072214609
:107280003846BDE8F04700F0E5BB00005824002078
:10729000D42200202DE9F04F0746858802883D481A
:1072A000012197B08346102A09D0112A49D01A2A01
:1072B0006CD1387AB1EB101F45D2012244E0354C35
:1072C000083CA068C0430B9061680BA801F0AFF8C0
:1072D0000B990CA800F058FB2C220CA96846FFF76C
:1072E00031F80026E946A04610E000BF09EB460051
:1072F0005FF00004B0F804A008EB84005146001DC4
:1073000001F069F8641C1D2CF6D3761C0098B0427D
:10731000ECD8142D05D317B00420BDE8F04FFFF7CB
:1073200035BC2946584601F06CF8294608F104009E
:1073300001F067F8F87B012828D016482946001D7F
:1073400015E029461AE000220221B1EB101F01D2FC
:10735000012600E000260F49083901F11000041D44
:10736000294682B101F04DF836B12946204617B0C2
:10737000BDE8F04F01F045B82946204617B0BDE8FA
:10738000F04F01F028B801F026F8F5E717B0BDE896
:10739000F08F00007C24002030B58DB004462E4BC9
:1073A000086860610FCB08AD85E80F0004F1120199
:1073B00008A862DF00284CD1A07C8DF8320041F291
:1073C0002350ADF8300022460CA90120A8DF002888
:1073D0003FD120216846FEF7CEFF41F22450ADF8A0
:1073E0000000A07C8DF8020001259DF80D00ADF88D
:1073F000065040F012008DF81150ADF804508DF891
:107400000D008DF81350208804F10A02694600F03F
:107410007BF900281DD120216846FEF7ACFF41F220
:107420002550ADF80000A07C8DF802009DF80D00FD
:10743000ADF8065040F00A008DF81150ADF8045038
:107440008DF80D008DF812502088A21C694600F0BE
:107450005BF90DB030BD000068AC020030B40288AA
:10746000502A10D1034630F8062F4C88A2420AD188
:107470004289012A07D14C69002C04D0027B9888EC
:10748000A44630BC604730BC704707B586B00122C7
:1074900000230093ADF810200193029303938DF81D
:1074A00002204989ADF8001008A9039104A90291AE
:1074B0006946AEDF09B000BD007800F001007047FA
:1074C0002DE9FC410646C0074FF000050ED0104FD5
:1074D00000240122385D009500231146019501F03A
:1074E000D5FA641C042CF4D300F024F8B0070DD5B1
:1074F000074E0024361D0022305D032300951146FF
:10750000019501F0C3FA641C042CF4D3BDE8FC819E
:1075100048AC02000249085C012101F048BB0000B0
:1075200048AC02000249085C002101F040BB0000A9
:1075300048AC020010B500242046FFF7EBFF641CA6
:10754000042CF9D310BD00002DE9F8430546861C34
:1075500000208DF8000090460F464FF00109684664
:10756000FFF7B0FB1B4C20683860D4E90001401ADB
:10757000A16804F21C47081A0EE00121384600F009
:1075800050FF00F033FD0146384600F04AFFD4E9D1
:107590000001401AA168081A401C8642EDD8B8F1D3
:1075A000000F03D0052065F3891002E0062065F383
:1075B0009F50A2682168114004EB8101C8602068D7
:1075C000304420609DF80000FFF7A0FB4846BDE86E
:1075D000F88300008828002070B50D4604460A296B
:1075E00002D10D21FFF7F8FFA0682268411CA160BD
:1075F0001554D4E90101814204D32046BDE870400E
:1076000001F04BB970BD0000034803C8814201D1AD
:1076100001207047002070478828002010B50C46D4
:107620000D281BD110481149401AC008032101EB55
:1076300000400FA101F0E4FC1548224613494088A0
:10764000FFF723FF00280DD0A0F54051023909D0E3
:10765000082807D043F20141884203D0BDE810401A
:10766000FFF794BA10BD0000DCB602009CB6020021
:1076700053656E6420627574746F6E2073746174E8
:1076800065206368616E67652E000000AC230020F2
:10769000B822002005494FF0FF32082841F8202089
:1076A00002D3084480F848207047000000250020DD
:1076B000F0B54FF0FF3512B10023082601E0082392
:1076C0000C260C4C05E000BF54F823707F1C04D03E
:1076D0005B1CB342F8D32846F0BD26185DB286F88D
:1076E000305044F82310002AF5D1E11881F8480001
:1076F000F1E70000002500200249084490F930001D
:1077000070470000002500202DE9F043814688786D
:1077100091B090460C4600B901208DF83E002088BB
:10772000ADF83C0000250095607C694602F05AFEE9
:107730006E46A07C711C02F055FEE07B00289DF88F
:10774000020002D040F0080001E020F008008DF8AF
:107750000200217C11B140F0100001E020F0100087
:107760008DF80200217B11B140F0010001E020F012
:1077700001008DF80200217D09B1022100E0012104
:1077800061F342008DF802001C2102A8FEF7F3FD10
:10779000607BC10601D4800617D50E950EAFE07C44
:1077A000791C02F01FFE9DF83800079720F00F00AB
:1077B000401C20F0F00010308DF838009DF83A00A1
:1077C00020F00600801C8DF83A00607B8DF80800E0
:1077D000A07B8DF80900142109A8FEF7CCFD0FA8A5
:1077E000CDE90906A088ADF83000A06820B1E08896
:1077F000ADF82C00A0680D90A06998B301950088A1
:10780000ADF81000A06901AD01A94088ADF81200E3
:10781000A069406806950390A069007B02F0E2FD34
:10782000A069691C407B02F0DDFDA069807A002818
:107830009DF8060002D040F0080001E020F00800AA
:107840008DF80600A169C97A11B140F0100001E07D
:1078500020F010008DF80600A169097A19B140F0F6
:10786000010002E00DE020F001008DF80600A169A2
:10787000897B09B1022100E0012161F342008DF80A
:107880000600E06900B10590434609AA02A94846EE
:10789000AADF11B0BDE8F08370B5084C050009D02F
:1078A00010342168002907D00868206049682846FC
:1078B0008847F6E70834F4E770BD0000EC240020A8
:1078C000054A012120B1012805D19170FFF7E4BFDD
:1078D00051700020FAE77047EC2400202DE9F05F9A
:1078E00026484168F1B3DFF898B00E688146DBF8AE
:1078F000004087688078E11B21F07F45ED1CB0B91E
:10790000DFF880804FF48030C8F84403C8F80403DF
:107910001120FEF707FE1120FEF70FFE4FF0010ABF
:10792000C8F800A02F2001F091FF89F802A0B5420D
:1079300000D23546124BE8193C3320F07F401860E6
:10794000DBF800105A46091B21F07F41001B20F094
:107950007F40C91C81420FD9106818602F2001F0A8
:1079600075FF00E004E0BDE8F05F1120FEF7F0BD18
:10797000BDE8F05F02F026BCBDE8F09F18230020B0
:10798000041501400010014073B58CB0064600207C
:1079900000900D9880B100246D4621460DA800F09E
:1079A00025FD30B1009805EB400084800098401C14
:1079B0000090641C142CF0D32C2269463046FEF74C
:1079C000C1FC0EB070BD2DE9F04117880646B81D08
:1079D00014460D46984202D90C20BDE8F08131884A
:1079E000072206290AD34FF4486C4FF6FF7361450E
:1079F00001D9994202D17088062801D21046ECE7DD
:107A0000604501D99842F9D1994203D0984201D0FA
:107A10008142F3D80520E85520881221401C80B20D
:107A2000208029542088401C80B220804119308851
:107A300002F0E3FF2188084480B220804119708859
:107A400002F0DBFF2188084420800020C5E7FFF713
:107A50009DB8000038B54A7A0F4B62B100220A7215
:107A60005969002906D001228DF80020ADF80200E6
:107A70006846884738BD0A7A62B19B684C680246FE
:107A800019462046FFF7CAF80028F3D0BDE8384071
:107A900002F03CBC5B68F1E75824002070B588B068
:107AA0000646002005900690ADF81410ADF81610AB
:107AB0000190029001AA05A9304690DF050021D06F
:107AC00001F06AFE0346114811493246401AC108C6
:107AD000012000EB014004460E4901F09CFABDF87C
:107AE000042012B9BDF8060028B1BDF806302046C2
:107AF00009A101F090FABDF808201AB120461649F4
:107B000001F082FA08B0284670BD00009CB6020061
:107B10009CB602006CAF02005468652072657175F6
:107B200065737465642054582F5258207061636BDC
:107B30006574206C656E67746820697320746F6F5C
:107B4000206C6F6E672062792025752F2575206F58
:107B500063746574732E0000B8AF02002DE9F0471E
:107B60000025DFF890803DE06068002100EBC5064D
:107B7000012032789146FEF7D1FBD4E9062300EAD2
:107B8000020701EA030C57EA0C0729D082438B4312
:107B90004846C4E9062301F03FFF32788246914609
:107BA00001200021FEF7BAFBD4E9042300EA020415
:107BB00001EA03074A4650460021FEF7AFFB444066
:107BC0004F403C430CD17078012801D0012000E0E7
:107BD0000020726880EA0A0012B1C1B2484690479C
:107BE0006D1CEDB298F8000044468542BCD3BDE858
:107BF000F0870000F822002010B50021024800F0B4
:107C000021FC80F3100010BDA42C00200E4910B5FB
:107C10000A784C780023A24212D0521CD2B20A70C9
:107C2000022A00D10B70084A0B780C3252F823203C
:107C300002608868104420F07F408860012010BDF9
:107C40000360002010BD0000182300202DE9F04142
:107C50008046024601200021FEF760FB1A4F0546D0
:107C60000E467868FFF71EF800280CD1174CD4E9AF
:107C7000062110462A4001EA06031A4305D0A8430C
:107C8000B143C4E90601BDE8F081404601F0C4FEFD
:107C900030B1D4E9040128433143C4E9040105E0CB
:107CA000D4E90410A943B043C4E90410D4E906019F
:107CB00028433143C4E90601A1687868BDE8F04172
:107CC0000022FEF7ABBF000084AC0200F8220020C7
:107CD0000146034802888A4200D000207047000015
:107CE000442400202DE9FC5F0E008346DDE90C47AB
:107CF000C6F1000098469246814600D40846012508
:107D000003E000BF90FBFAF06D1C5045FADAA8457D
:107D100000D9454624B1002E01DB780700D5641E4A
:107D2000B80702D5B8F1000F0AD0F80708D13CB166
:107D3000A54205D220215846641EFFF74DFCF6E708
:107D4000002E02DA4E462D2102E0780703D52B21C2
:107D50005846FFF741FC07F0030002280BD1B8F1A9
:107D6000000F08D13CB1A54205D230215846641E0F
:107D7000FFF732FCF6E7CDE900474346524631466D
:107D8000584602F03FFEBDE8FC9F000070B50D466E
:107D9000044600684FF4887101F01EFD4FF49071A5
:107DA000206801F019FD4FF49271206801F014FD74
:107DB0004FF4A271206801F00FFD20681149C0F84E
:107DC00004132068690740F30730090E002806DA1B
:107DD00000F00F0000F1E02080F8141D03E000F136
:107DE000E02080F800142068012140F3073000F003
:107DF0001F0291404009800000F1E020C0F800110E
:107E000070BD0000100302000246002012685307F4
:107E100013D502F00300012802D002280CD105E09E
:107E2000C2F383100B68801C184404E00223086826
:107E300003EB92521044086001207047F0B584882B
:107E4000A518944200D82246A41AC288D6189A428D
:107E500000D81346D21A4B880788BB420CD34088FF
:107E6000834209D88888A04206D3A84204D8C8888B
:107E7000904201D3B04201D90020F0BD0120F0BDF5
:107E80000B480C4910B5401AC008032101EB00440F
:107E90004FF0020022B1FFF745FB204606A103E0A8
:107EA000FFF738FB204609A1BDE8104001F0A8B853
:107EB000DCB602009CB602005265636569766564B3
:107EC000204C4544204F4E21000000005265636560
:107ED00069766564204C4544204F464621000000E9
:107EE0001721018041800021017141711B218171A5
:107EF000C17170472DE9F047394E002780463D4655
:107F0000DFF8E090D6F804A057E003D00446D0F89C
:107F10001C8035E099F8002002EB4201521CD2B2DD
:107F200089F8002009EBC10199F80230091D9A4235
:107F300001D189F8005048680A780446012A12D015
:107F4000022A02D0032A3BD108E002F03FFB00B135
:107F50000127257434E00574C06900E070680028CA
:107F6000F9D170602CE0207C50BB88686060C868E4
:107F7000A0600869E0604869A061F07800B16560C0
:107F80006268B168184B501A20F07F40984202D2C4
:107F9000A168084406E0881AA16820F07F40814269
:107FA00002D9081A206000E0256065600120A56004
:107FB00020742046E56102F0EBFAB8F10000A4D18C
:107FC00099F8001099F801008142A3D117B971689E
:107FD000514502D00120BDE8F0870020FBE70000FA
:107FE00018230020CC250020FFFF7F002DE9FF4152
:107FF0000026234800F012FA2148001F074600F02F
:108000000DFA204C60680090A56800E00098694671
:10801000284004EB80000C30FFF7F6FE0028F5D175
:1080200001AA009901EA050304EB8303491CDB68FC
:1080300042F82030401C00910228F2D3019800F051
:10804000030001280BD0022810D10198032101EB75
:1080500090500099BDF80A6001EB900005E001988E
:10806000BDF80A60C0F3831008440090384600F061
:10807000D2F908B10098606004B03046BDE8F081E4
:10808000A02C00208828002088B04FF40041002058
:1080900001F022F808B1FEF779FD00F089FE012019
:1080A000FFF70EFAFEF790FD08B1FEF76FFD40F204
:1080B000666201214748FEF7EBFC08B1FEF766FD5A
:1080C00001F020F908B1FEF761FD01F0B1FA08B145
:1080D000FEF75CFD002469460120009401F062F97E
:1080E00008B1FEF753FD684601F0DCF908B1FEF770
:1080F0004DFD9DF8080038A120F00F00401C20F035
:10810000F00010308DF808000D2202A87CDF08B1C5
:10811000FEF73CFD00945020ADF80000A020019433
:10812000ADF80200ADF804404FF4C870ADF8060099
:1081300068467ADF08B1FEF729FD00212A4800F0E1
:10814000F6F908B1FEF722FD284801A9CDE9004063
:108150002548143000F0AFFA08B1FEF717FD2448A7
:108160000090214869461838FFF716F908B1FEF764
:108170000DFDFEF701FC1C216846FEF7FCF84FF4EC
:108180002020CDE90040801002901A480590032578
:1081900019488DF80C500690ADF80E408DF810403F
:1081A0006846FEF717FF08B1FEF7F0FC13481449C4
:1081B000401AC00805EB004012A100F021FFFEF7B5
:1081C0002DFC00BF00F002FE0028FBD101F0AEF84C
:1081D000F8E70000BC2200204E6F726469635F42C2
:1081E0006C696E6B79000000C4230020719302005B
:1081F000817E0200399F02004F7A0200DCB6020045
:108200009CB60200426C696E6B79206578616D7076
:108210006C6520737461727465642E0070B51446C9
:1082200082880E4605462088111D0144921C994201
:1082300001D8FE2A01D90C2070BD521C325420886E
:10824000FF21401C80B2208031542088401C80B225
:1082500020808119288802F0D0FB2188084480B250
:108260002080AA8842B1A96841B13044FEF76AF87B
:108270002088A98808442080002070BD072070BD98
:108280002DE9F047C5881E1DB6FBF5F78946B6FBFC
:10829000F5F1044605FB176C407916686843DDF874
:1082A00020A0F718001F874200D9C61A166001E007
:1082B0002468491E0029FBD1A5EB0C078846B7426C
:1082C00016D818E004EB0C00001D09EB0803BAF106
:1082D000000F3A4602D00146184600E01946FEF764
:1082E00031F82468F61B4FF0000CB844B54201D9B0
:1082F000374600E02F46002EE4D1BDE8F0870000AD
:1083000030B5024651B100F005FF0021074C08E0EE
:1083100034F821301568AB4202D11160002030BD25
:10832000491C8142F4D3052030BD0000000000004C
:10833000F8B50F46017814460546012901D1687841
:1083400030B12088821C9A4232D8012902D006E03E
:108350000720F8BD69780144891C994228D8181A69
:10836000801E86B2ADF800602188B81C08446946BA
:108370007DDF0028EDD12978022904D06878BDF886
:108380000020904205D3BDF80000B04201D809207A
:108390000AE00820012905D16978B14202D8ADF878
:1083A000001001E0ADF80060BDF80010FE2901D911
:1083B0000C20F8BD2288491CB9542188491C89B277
:1083C000218078542088401C2080BDF8001008448B
:1083D00020800020F8BD01F01F0301229A40D24303
:1083E000490900EB8100114600F021B84A0950F814
:1083F000220001F01F0201219140084000D001201D
:10840000704701F01F0301229A40490900EB8100E7
:10841000114600F01CB8002100F00FB8012100F057
:1084200016B808B56A46FDF728FF009808BD08B5DC
:108430006A46FDF708FF009808BD08B56A46FDF7D3
:1084400002FF08BD08B56A46FDF7E4FE08BD08B5A1
:108450006A46FDF7EBFE009808BD08B56A46FDF7D1
:1084600019FF009808BD38B5044600258DF8005066
:108470006846FEF727FC21686268086890420ED9BA
:10848000401E08600178238AE26801FB0325227AF6
:108490002168101AC0B20A79824200D208719DF890
:1084A0000000FEF733FC284638BD38B505460020ED
:1084B0008DF800000C466846FEF704FCE868298A3F
:1084C000201AB0FBF1F12A681068431C1360017098
:1084D0009DF80000FEF71AFC38BD10B530B1017AE6
:1084E00042680368891AC9B21A6006E00E2010BDFE
:1084F00003681A68541C1C601170491EC9B2F7D277
:10850000006800210171084610BDC20800F0070391
:108510000120895C98400840704710B5C20800F0FF
:108520000703885C01249C402043885410BD10B58B
:1085300060B10161172120F8021B20F8021B1B21EA
:1085400000F8021BFFF7CCFC002010BD0E2010BD70
:10855000F0B5858893B00C46002D39D101880026EE
:108560003F4F24293BD006DC102909D011290CD01B
:10857000232958D14FE03A290BD0552953D129E06E
:108580000146204601F0E6FC4DE0A01DFFF7A8FCE7
:1085900049E02246408934F8061F814200D8084647
:1085A0006080172800D217206080106970B1607950
:1085B00060B1D7E90001CDE90301ADF80E50608844
:1085C000ADF81000136903A910469847667126712B
:1085D00013B0F0BD0146204601F010FD23E0011D5F
:1085E0002C2206A8FDF7AEFEBDF81800BDF81C2031
:1085F00004EBC0014A732269AAB1D7E90423CDE98B
:108600000423ADF81200487B8DF81400226920463F
:1086100004A9904707E0017A207B884200D20146F6
:108620002846FFF73BFAA07A0028D1D0E1882846F7
:10863000A5DF012580B11128CAD001F0ADF80246AE
:108640000848094913B0401AC00805EB0040BDE8CE
:10865000F04006A100F0D8BCA672E572B8E70000B1
:1086600050AC02009CB602009CB6020073645F62CC
:108670006C655F67617474635F65786368616E677A
:10868000655F6D74755F72657175657374282920F7
:1086900072657475726E65642025732E000000008B
:1086A00020B10278DE2A03D0082070470E207047E0
:1086B00041800020704760B159B10278DE2A0AD0AB
:1086C00009684160DE2101704FF6FF714180002092
:1086D00070470E207047082070477FB50546002977
:1086E0004DD0002D4BD008780C46DE2847D1A88805
:1086F0006188884202D1204602F012FA28880128B7
:1087000025D002283BD011283AD0512837D135F84E
:10871000040F6188884232D1A978A81C02292ED181
:10872000017A042903D0062901D0052927D1002187
:10873000009102228DF8002001914FF4C072029145
:108740000391ADF80420007A05280FD010E0297AB3
:108750002046012913D1A988428891420FD10121D5
:10876000017204B0BDE8704002F0DAB9ADF804104F
:1087700028886946B0DF002801D0616888477FBD3E
:10878000A88861888842FAD14FF6FF7060807FBD6B
:1087900000F180400068002800D00120704708B533
:1087A00000F18040002101600068009008BD0000D9
:1087B00070B50B4C207808B185250FE00020A06033
:1087C00060602061E060074801F022F8054600F093
:1087D0007BFF08B901F006F801202070284670BD23
:1087E000EC240020C178020038B500258DF8005037
:1087F0006846FEF767FA074CE068401EE060E068F4
:1088000010B901F015F8A5709DF80000FEF77EFA8A
:1088100038BD0000EC240020F0B50546047815486A
:1088200089B0164640F82420124A0869121DA2F1A8
:10883000080742F82400487F385520226846FDF793
:1088400081FD04942878385C48B10EB10A4A00E0F2
:1088500000226946281D01F08BFA09B0F0BD0EB167
:10886000064A00E00022694605F10C0001F054F9C7
:10887000F3E70000E0220020D9A8020025A70200AB
:108880000FB408B50399002904D004AA00926A46DF
:1088900000F00FF801B05DF814FB10B582680446D3
:1088A000002A05D0D4E90403216898470020A0607D
:1088B00010BD2DE9FC4791460C00804676D014F897
:1088C000011B39B125290ED04046FEF785FE2078E0
:1088D0000028F4D198F80C00002867D04046BDE885
:1088E000FC47FFF7DABF0020012221782B291BD09B
:1088F0002D2902D0302908D102E040F0010001E02A
:1089000040F00200641C002AEFD100252A290ED075
:108910002178A1F130020A2A11D205EB850201EB80
:108920004205641C303DF1E740F00400EAE7D9F865
:1089300000100B1DC9F800300968641C0D44217833
:1089400000232E290BD114F8011FA1F130020A2AAD
:1089500005D203EB830201EB4203303BF3E76C29C2
:108960000DD068290BD0692921D00BDC252918D01E
:10897000582931D063290ED0642915D117E014F895
:10898000011FECE7702969D0732932D075291BD0FB
:10899000782909D120E0D9F80000011DC9F800109C
:1089A00001784046FEF718FE641C90E76CE0D9F8A9
:1089B00000100A1DC9F800200968CDE900500A22FC
:1089C0004046FFF78FF9EFE7D9F800100A1DC9F804
:1089D000002009680A2206E0D9F800100A1DC9F82B
:1089E000002009681022CDE90050404602F00AF844
:1089F000DAE7D9F8001000270A1DC9F800200E6830
:108A0000C00705D112E04046761C7F1CFEF7E4FD4E
:108A100031780029F7D104E0202140466D1EFEF791
:108A2000DBFDBD42C0D9002DF6D1BDE74EB13046C9
:108A3000FDF7ACFC074604E0202140466D1EFEF722
:108A4000CBFDBD4206D9002DF6D103E04046761C91
:108A5000FEF7C2FD31780029F8D1A5E7D9F800006A
:108A6000011DC9F80010056830214046FEF7B4FD2D
:108A700078214046FEF7B0FD08200021CDE9000135
:108A8000034610222946B0E7BDE8FC8770B541EAED
:108A90004201DDE904564FF0A04441EA830141EA76
:108AA000052104EB800041EA0641C0F8001770BDC3
:108AB00070B541EA4201DDE904564FF0A04441EAB5
:108AC000830141EA052104EB800041EA0641C0F838
:108AD000001770BD70B541EA4201DDE904564FF060
:108AE000A04441EA830141EA052104EB800041EA08
:108AF0000641C0F8001770BD70B541EA4201DDE9DA
:108B000004564FF0A04441EA830141EA052104EBF9
:108B1000800041EA0641C0F8001770BD1CB5002175
:108B200000910B4601220191FFF7D4FF1CBD1CB53B
:108B3000002100910B4601220191FFF7DDFF1CBDD2
:108B40001CB500220B46009211460192FFF7C2FFAE
:108B50001CBD1CB500220B46009211460192FFF786
:108B6000CBFF1CBD1CB5002100910B4601220191D9
:108B70001146FFF7AFFF1CBD1CB5002100910B464D
:108B8000012201911146FFF7B7FF1CBD4FF0A04233
:108B900002EB8000D0F8002722F44032C0F8002712
:108BA000D0F8002742EA0141C0F8001770470122BF
:108BB0004FF0A043824011B1C3F808257047C3F8B5
:108BC0000C25704718B5084B6C4601441B68009390
:108BD00006E000BF54F82030D3F81035401C08C21E
:108BE0008142F7D818BD000078AC0200034908B5EF
:108BF0000844002101600068009008BD006000404A
:108C000002494058012800D0002070470060004011
:108C100030B5154A01460020D2F8104423460AE038
:108C2000DB681D79854205D1401C0A28F6DB4FF030
:108C3000FF3030BD1B68002BF2D1431CF9D0CB684C
:108C40001871D2F8103443B1DB68CC681B6823601C
:108C5000D2F81024D268116030BDC2F81014C9686F
:108C600000220A6030BD000088280020F0B595B0D1
:108C70001C4615460F4608461A9E00F01DFB18219B
:108C800009A8FDF778FB0E96CDE9095400230822C8
:108C900003A9384600F025FB05980690BDF81000A2
:108CA000ADF81C00BDF81200ADF81E0000208DF8D4
:108CB00021000398082600F00300012802D00228B2
:108CC00018D032E003983346850AC0F3C2008DF80D
:108CD000200003980FA9C0F38314A200384600F0C7
:108CE00000FB09A8009006AB22460FA9284600F019
:108CF0003FFA1AE00398840DC0F3C2008DF82000FB
:108D0000082C01D2254600E0082533462A460FA943
:108D1000384600F0E6FA2E44641B09AB06AA294641
:108D20000FA800F081F9002CEAD1384600F0CAFA09
:108D300015B0F0BD7047012001F012BD084810B514
:108D40000178084A515C19B1001D01F09DF802E05C
:108D50000C3000F0ABFFBDE81040002001F000BD7A
:108D600038230020DC22002008B5034A009240236B
:108D7000024AFFF77BFF08BD1DA30200F02600207A
:108D80000A4A012902EBC00007D0022907D00329B3
:108D900007D0042907D00020704702207047042024
:108DA0007047007970474079704700009CB6020018
:108DB00010B5FFF7C0FF04210348FFF729FF024960
:108DC0000120C968487110BD8CB602002DE9F04F32
:108DD0008DB0FEF719FC18B100200DB0BDE8F08F82
:108DE0007E4C4FF0000BC4F818B4BFF34F8F60688F
:108DF0000290A568D846284004EB80000CE000BF34
:108E0000D4F8180470B921680298814201D86160D1
:108E1000E2E7284004EB80000C3002A9FEF7F4FFE3
:108E20000028EDD1002005AA029901EA050304EB10
:108E30008303491CDB6842F82030401C0291022861
:108E4000F2D3059800F00300022802D001284DD08B
:108E5000AAE005985022810D8946B2EB905F00D8B8
:108E600050210E4666F39F50059008315C4800F093
:108E7000DAF9070078D000F01FFA4346082205A966
:108E8000384600F036FA029908F1080A2940681AB3
:108E90008000001D864222D9504D0C3530B1C2B23F
:108EA00004EB8101301A90460C3104E02946F2B2FD
:108EB000002590462846C6B25346384600F019FAB7
:108EC0000AEB080325B132462946384600F011FA6C
:108ED000029909F1030001EB900002903BE004EBE2
:108EE00081015346324638460C31EFE70598C0F30E
:108EF0008310062800D30620059960F38911C1F379
:108F00008310801C05918100354800F08CF9070022
:108F10004AD000F0D1F94346082205A9384600F0AE
:108F2000E8F908F1080800260FE00298434600EA35
:108F30000501401C04EB81010290042238460C31EB
:108F400000F0D7F908F10408761C0598C0F38310E7
:108F5000B042EAD847B1D4F81054D4F8180478B124
:108F6000384600F0AFF934E01EE0E86840790128A7
:108F700004D12A682846394612689047E86805688F
:108F8000002DF2D1384600F09DF98DF800B068460A
:108F9000FDF798FED4F8180408B9029860609DF8AF
:108FA0000000FDF7B3FE14E0D4F8104405E021689A
:108FB000204689688847E0680468002CF7D1094892
:108FC0000949401AC008022101EB004007A100F046
:108FD00017F8FEF719FB80F00100FEE68828002054
:108FE000FCB60200DCB602009CB602004261636B74
:108FF000656E647320666C757368656400000000BC
:1090000000231A4601F03EBA08B5012300926A46D1
:1090100001F038FA08BD1CB5CDE9002302236A46E9
:1090200001F030FA1CBD00002DE9F0470E468046E5
:109030001C469246082940D894F80C9000202073D2
:109040001946104601F066F80025B54206D218F818
:1090500005201BA12046FFF713FC03E01AA12046C0
:10906000FFF70EFC6D1C082DEFD318A12046FFF76B
:1090700007FC0025B54212D218F805707E2F08D8DB
:10908000FDF75CF90068C05D10F03E0F01D03A4674
:1090900000E02E220EA12046FFF7F2FB03E00DA117
:1090A0002046FFF7EDFB6D1C082DE3D3012221467E
:1090B000504601F011F884F80C90BDE8F0870000EC
:1090C0002025303278000000202020007C000000A5
:1090D00025630000200000000B4810B5FF218160CF
:1090E000002101604160C0F81814C0F8141480F821
:1090F0002014064800F0E4F8002803D1044800F0EA
:1091000039F9002010BD000088280020FCB60200BC
:1091100034AE020002480349401AC00870470000FC
:10912000FCB602009CB6020013B56846FFF7E8F8EB
:1091300008B100201CBD0248009950F831001CBD48
:109140009CB6020070B509480125D0F8104480F89B
:10915000205407E0E0684571216820464968884747
:10916000E0680468002CF5D170BD0000882800205C
:109170002DE9FF4781460C9D00200C462F7B28736C
:10918000984616462946184600F0C4FF072E42D2DC
:10919000DFE806F004090F161F2A36004946284664
:1091A000FFF76EFB37E0494628462268FFF768FB69
:1091B00031E0D4E9002349462846FFF761FB2AE065
:1091C000A0680090D4E9002349462846FFF758FBE1
:1091D00021E0D4E90201CDE90001D4E900234946A8
:1091E0002846FFF74DFB16E004F1080007C88DE89C
:1091F0000700D4E9002349462846FFF741FB0AE06F
:1092000004F108000FC88DE80F00D4E90023494697
:109210002846FFF735FB00222946404600F05CFF58
:109220002F73BDE8FF872DE9F041058A80462D1F89
:109230004819C01CB0FBF5F0C6B24046FFF713F961
:10924000041E19D00020207101206071E5800027E4
:109250002546761EC4F800800BE04046FFF703F970
:1092600060B16179491C6171286005467F1CC0F8B6
:109270000080B742F1D32046BDE8F081204600F0DF
:1092800002F80020F8E72DE9F041457901466B1E10
:10929000002201E00968521C9A42FBD30F68014684
:1092A000002605E038460C68FFF7FFF82146761CDB
:1092B000AE42F7D3BDE8F0810121001DFFF7B1B840
:1092C000FFF70BB910B504460121001DFFF7C5F8E3
:1092D00010F0FF0F04D12046BDE81040FFF7D3BFC8
:1092E00010BD1CB501920122009201AAFEF7C8FF31
:1092F0001CBD1CB501920022009201AAFEF7C0FF1E
:109300001CBD0000064910B500204870091D08600A
:10931000BFF35F8F0349044800F0FAF9002010BD45
:109320002C230020C0AC0200E426002008B5002059
:109330008DF800006846FDF7C5FCF1EE100A20F03C
:109340009F00E1EE100ABFF35F8F08494020C1F88B
:1093500080029DF80000FDF7D9FC00F0B5F908B1D6
:1093600041DF08BD20BF40BF20BF08BD04E000E0D2
:10937000FDF70CBC826800219160826811618268EF
:1093800051618268D1608268516080680160704775
:1093900020B1034909680160002070470E20704722
:1093A000B8AE0200FEB502460E460846FFF7F0FFD3
:1093B000002868D1002400940194012706208DF82C
:1093C0000020ADF8040002948DF802706946202058
:1093D000326869DF2C492D4A891AC908012202EB3B
:1093E000014530B100F0D8F9024628462849FFF778
:1093F0000BFE00948DF801708DF8024001940294E8
:109400008DF8034069464020326869DF30B100F0D2
:10941000C3F9024628461F49FFF7F6FD00940A20CB
:109420008DF800000194029469460120326869DFDA
:1094300030B100F0B1F9024628461749FFF7E4FDC4
:109440004FF4B0600090019402946946A120326804
:1094500069DF30B100F0A0F9024628460F49FFF756
:10946000D3FD0094019402948DF800406946A02039
:10947000326869DF30B100F08FF9024628460849AA
:10948000FFF7C2FD0020FEBDECB602009CB6020054
:1094900058B50200A0B50200B8B4020004B502003D
:1094A00064B402002DE9F0410546076860DF80469C
:1094B00019491A482A68081AC608BA4219D9022056
:1094C00000EB064416A12046FFF79AFD20463A46D7
:1094D0001FA12B68FFF79FFD4FF08050D0F80C01C3
:1094E0002968800200F10050421A204625A1FFF7AA
:1094F0008BFDB8F100004FF001040AD000F04CF9E8
:10950000024604EB06402AA1FFF77EFD4046BDE877
:10951000F0812F480470F9E7ECB602009CB6020017
:10952000496E73756666696369656E742052414D54
:1095300020616C6C6F636174656420666F72207467
:10954000686520536F66744465766963652E000014
:109550004368616E6765207468652052414D2073D1
:1095600074617274206C6F636174696F6E206672CF
:109570006F6D203078257820746F20307825782E14
:10958000000000004D6178696D756D2052414D20DD
:1095900073697A6520666F72206170706C696361AF
:1095A00074696F6E20697320307825782E00000072
:1095B00073645F626C655F656E61626C652829200B
:1095C00072657475726E65642025732E000000004C
:1095D000A723002030B5144891B00078002820D08F
:1095E0005FF03405ADF8405010A903A861DF30B139
:1095F000052816D011B0BDE83040FDF7C7BA03AC5E
:109600000A49684600F084F807E000BFD0E900216D
:1096100020469047684600F092F802980028E1D072
:10962000F4E711B030BD0000A7230020BCAE02005B
:109630007CB5194C207808B108207CBD0120A070B1
:10964000002000F035FE112819D0002000F048FE5F
:1096500012480026006801908DF800606846FDF70A
:1096600031FB0F4901A810DF05000AD0002020704F
:109670009DF80000FDF74AFB2DB128467CBD002077
:109680007CBD0120F3E7A670667000F0CFFE0120DC
:1096900000F026FEF3E70000A423002050AE0200F5
:1096A000096B02000EB50749684600F031F805E085
:1096B000D0E900108847684600F041F80298002879
:1096C000F6D10EBD6CAE0200014800787047000074
:1096D000A42300201FB568464BDF30B1052814D005
:1096E00004B0BDE81040FDF751BA084901A800F0E8
:1096F0000FF806E0D0E900210098904701A800F09B
:109700001EF803980028E6D0F4E71FBDD8AE02008B
:10971000016009684160AFF3008010B5D0E9002115
:109720005368994201D1002104E0D1E90034A342F9
:1097300002D01946816010BD08314160F0E78168B0
:1097400000290BD0026892680A44826041684B6825
:109750009A4203D108314160FFF7DFBF7047000034
:109760000C4A10B502F594730EE0991AC91001EB7A
:10977000D171491002EBC1010C68844201D90B463A
:1097800002E005D201F108029A42EED3002010BD9A
:10979000486810BDE0AC020000B5FFF7E1FF00280B
:1097A00000D1014800BD0000CCAC020040580028A8
:1097B00000D00120704708B5002242504058009068
:1097C00008BDD0F80403084000D00120704740587D
:1097D000002800D00120704708B5002242504058B0
:1097E000009008BD08480068012110F0010F06D163
:1097F0004FF0E020C02280F80024C0F80011034997
:10980000012008607047000000E100E018050040FA
:109810000649024600200B790BB1852070470A608B
:1098200001220A7100224A7170470000E8220020DC
:1098300004490120086004480168C1F3004100297F
:10984000FAD170470C00004018040040002802D0F4
:10985000014980010847704791AC020010B50446E9
:1098600000F022FC28B12046BDE810400021FFF79F
:109870008DB9204600F024FC00280FD02046FDF7CB
:109880003BFF074A02EB8001D1F8103523F00103BA
:10989000C1F8103501218140C2F8081310BD000045
:1098A000006000402DE9F0418846054600F0FCFBD1
:1098B000234E002828461AD0FDF71EFF304490F8AA
:1098C00048008009032802D001280ED007E04FF09D
:1098D000A040D0F81005E84010F0010F05D003219A
:1098E0002846BDE8F041FFF751B90221F8E700F042
:1098F000E7FB002822D02846FDF7FEFE04464FF481
:10990000807000EB84000F4F81B207EB8400D0F829
:10991000102542F00102C0F810250846FFF766F94D
:10992000B8F1000F0AD02846FDF7E6FE56F82000F1
:10993000002803D00120A040C7F80403BDE8F0814F
:1099400000250020006000402DE9FC41DFF8BC80CC
:10995000044608EB0400002790F930001346C017B6
:109960000E46401C01D008274CE0B0781946C0F3E1
:1099700040022046FDF79CFE0546401C41D0B078D1
:10998000410719D4C0070AD04FF0A04000EB840172
:10999000D1F8000720F00200C1F8000707E000211D
:1099A0007378204600910A460191FFF781F8174924
:1099B00020465431FEF7B1FDB078800718D5144821
:1099C000317800EB8500D0F81025124B1A40C0F812
:1099D00010254FF4F8524FF4403302EA042203EA10
:1099E00001410A43D0F810150A43C0F8102509E0D8
:1099F00008EB0500327810F8481F41EA8211017027
:109A000000E004273846BDE8FC8100000025002066
:109A100000600040FFE0FCFF4FF0A041D1F81015BE
:109A2000C14011F0010000D00120704770B5174D02
:109A300095F8580008B1082070BD0020411E2A1872
:109A4000401CC0B282F830102028F8D300242046F1
:109A5000FDF720FE641CE4B20C2CF8D300240C4962
:109A6000C0206C6581F8000401264020891FC1F8E0
:109A700000014FF4BE70FFF7B9F80649F007C1F8CE
:109A8000040385F85860204670BD000000250020C2
:109A900006E000E000600040034890F8580000280D
:109AA00000D0012070470000002500200121B1EB0B
:109AB000507F01D1012070470020704738B50D4616
:109AC00000F074FB040014D000208DF800006846FC
:109AD000FDF7F8F8207928B19DF80000FDF716F998
:109AE000112038BD0120256020719DF80000FDF790
:109AF0000DF9002038BD10B500F058FB002802D049
:109B000000210160017110BD0149024800F050BE02
:109B10005C250020002000402DE9F0410546007939
:109B200016460F4600EB40012C4A01EBC00102EB48
:109B3000810494F82A1011B10820BDE8F081284969
:109B400051F820102868FFF7B9FF08B11120F4E799
:109B500039462846FDF7F4F8666038692060300021
:109B60004FF001062DD03F7F4FF48E712868FFF72C
:109B700022FE4FF4A2712868FFF71DFE28681949DC
:109B8000C0F8041328684FEA471140F30730002853
:109B900006DA00F00F0000F1E02080F8141D03E069
:109BA00000F1E02080F80014286840F3073000F04E
:109BB0001F0106FA01F14009800000F1E020C0F821
:109BC000001128680421C0F800150020A061E061A0
:109BD00084F8290044F8140FA675AEE75C25002030
:109BE0007CAC0200800002002DE9F04705460079B8
:109BF0000B4600EB400101EBC000234901EB800460
:109C0000284600F043F810B11120BDE8F0874FF06E
:109C10000008C4F82080A360626184F828804FF4B3
:109C20008E76474631462868FFF7C5FD28684FF015
:109C30000109C0F808902146286800F055FD6068C9
:109C400000BBD5F800A00EE094F8280008B10F275B
:109C500016E031465046FFF7A9FD0028F4D0214612
:109C6000504600F041FD216A60698142F1D33146DE
:109C70002868FFF79BFD0028F9D02868C0F80C90F1
:109C8000C4F814803846C0E75C250020007900EB5A
:109C9000400101EBC000044901EB8000406900284D
:109CA00000D00120704700005C2500202DE9F0471E
:109CB000044600794FF0000900EB400101EBC000C1
:109CC000254901EB80072068C0F80095786880B1CD
:109CD00020682249C0F808132068012140F30730AA
:109CE00000F01F0291404009800000F1E020C0F820
:109CF00080112068D0F80C25D0F81485D0F80865BC
:109D0000D0F810554FF0FF31C0F81415C0F80C15FD
:109D10002068C0F80815C0F81015501C02D0104675
:109D2000FEF7FCFEB8F1FF3F02D04046FEF7F6FE1C
:109D3000681C02D02846FEF7F1FE701C02D03046A7
:109D4000FEF7ECFE2068FFF7D6FE87F82A90C7F8EA
:109D50000490BDE8F08700005C250020840202002A
:109D60000149024800F0D0BD8825002000200040B5
:109D70002DE9F0410546164600790F46154A00EBDD
:109D8000C00102EB810494F8201011B10820BDE855
:109D9000F081114951F820102868FFF78FFE08B1B3
:109DA0001120F4E739462846FDF70EF86660386959
:109DB00020601EB1397F2846FDF7E8FF286808219A
:109DC000C0F800150020A061E0616061012184F805
:109DD0002010DCE78825002080AC02002DE9F04748
:109DE00004460E460079204900EBC00001EB8005D7
:109DF00017463046FFF75AFE30B1204600F036F8DD
:109E000020B11120BDE8F0871020FBE76F61AE6044
:109E10004FF49076002731462068FFF7DDFC4FF4C1
:109E2000AC7841462068FFF7D7FC2068AA686969CA
:109E3000C0F84425C0F84815206801218160686891
:109E400078B9B14649462068FFF7C1FC064641464D
:109E50002068FFF7BCFC0643F4D000B10F270020B8
:109E600068613846CEE70000882500200079054962
:109E700000EBC00001EB80004069002800D0012009
:109E800070470000882500202DE9F047044600793E
:109E9000274900EBC00001EB800720684FF0000964
:109EA000C0F80095786880B120682249C0F808138E
:109EB0002068012140F3073000F01F029140400963
:109EC000800000F1E020C0F880112068D0F80C2557
:109ED000D0F81485D0F80865D0F810554FF0FF3150
:109EE000C0F80C15C0F814152068C0F80815C0F8A3
:109EF0001015501C02D01046FEF719FEB8F1FF3FB6
:109F000002D04046FEF713FE681C02D02846FEF73A
:109F10000EFE701C02D03046FEF709FE2068FFF7E7
:109F2000EAFD87F82090C7F80490BDE8F0870000AC
:109F300088250020100302000078002807D104487B
:109F40003B21408876DF002801D0FCF71FBE704718
:109F5000B822002070B58D88027900EBC504227309
:109F6000C97BA41D012902D0022904D101E0008887
:109F700000E04088208021886088814211D92846ED
:109F8000A5DF0126B0B1112816D0FFF705FC024667
:109F90000B480C49401AC00806EB00400AA1FFF725
:109FA00033F8A179E079814208D92846BDE87040AC
:109FB000FDF774BD6671F4E72671F2E770BD00002D
:109FC0009CB602009CB6020073645F626C655F67BA
:109FD000617474635F65786368616E67655F6D74F3
:109FE000755F726571756573742829207265747563
:109FF000726E65642025732E000000007CB5064655
:10A000008D88C88806EBC504A41D172800D2172028
:10A010002188814200D80846608000202071218874
:10A020002846B5DF60B1FFF7B7FB02460F4810497D
:10A03000401AC008012101EB00400EA1FEF7E4FF29
:10A040006079002810D1306900280DD01549D1E978
:10A050000201CDE90001ADF802506088ADF80400BE
:10A0600032696946304690477CBD00009CB60200CC
:10A070009CB6020073645F626C655F6761747473A1
:10A080005F65786368616E67655F6D74755F726543
:10A09000706C7928292072657475726E656420254C
:10A0A000732E000050AC02000449084490F93000BF
:10A0B000082801DB012070470020704700250020A0
:10A0C0000449084490F93000082801D20120704763
:10A0D000002070470025002010B50C46017A0529A4
:10A0E00008D0407A38B1084808A102682046FEF737
:10A0F000C7FB00E01AB106A12046FEF7C1FB2046CF
:10A10000BDE81040FEF7C9BB802300202573000086
:10A110000D0A000038B5C3880D46044633B114A0BB
:10A12000009015A216A12846FEF7AAFB217A052960
:10A130001CD0607A48B1A088FEF722FE164951F87B
:10A14000202016A12846FEF79BFBA0880021FEF7E1
:10A15000EBFF03461049207A143951F8202001B052
:10A160002846BDE830400EA1FEF78ABB38BD00008E
:10A170001B5B306D000000001B5B313B33316D0019
:10A1800025734C6F67732064726F7070656420284C
:10A1900025642925730D0A00802300202573000003
:10A1A0003C25733E2025733A200000000349884275
:10A1B00001D1034870470020704700000020004094
:10A1C000F022002070B5012670044FF0E021002538
:10A1D000C1F88001084C4010C4F84803C4F80803D3
:10A1E00066602F20FFF732FBA660044C2F20A5608D
:10A1F000FFF72CFBA57070BD001001401823002054
:10A2000070B5054688690C4600284FF484712846CD
:10A210000AD0FFF7D0FAD5F81805626AE1688854C9
:10A22000606A401C606270BDFFF7C5FAD5F818057A
:10A2300070BD1FB501238DF80030CDE90121D0E9B3
:10A240000012684690471FBD1FB501238DF80030EE
:10A25000CDE90121D0E90012684690471FBD0000FA
:10A2600038B50021012548B101280CD0032809D1B7
:10A27000FFF7B8FABDE83840FEF7B6BA4FF0E02075
:10A28000C0F8805138BD8DF800106846FCF71AFD03
:10A29000064C207808B9FEF78BFAE068401CE060B5
:10A2A000A5709DF80000FCF731FD38BDEC240020BE
:10A2B0003EB5044609496846FFF72AFA08E000BFA0
:10A2C000D0E900212046904730B16846FFF737FAC1
:10A2D00002980028F4D13EBD11203EBD54AE0200CC
:10A2E0003EB5044608496846FFF712FA07E000BF8A
:10A2F000D0E90021204690476846FFF720FA0298EF
:10A300000028F5D13EBD000060AE02000249896917
:10A31000002900D0084770475824002070B50D4C24
:10A320000020D2B22070201D0B4D0378EB5C1BB1D6
:10A33000001DFFF753FD02E00C30FFF755FC08B19C
:10A34000FCF724FC6078002802D021780029FAD09C
:10A3500070BD000034230020DC2200202DE9F041F4
:10A360000746806A14468846C8B3002531E000BF1E
:10A37000B96A05EB450001EB8006B088801CFE2819
:10A3800002D90C20BDE8F0812288401C08F80200A8
:10A3900020881622401C80B2208008F800202088E7
:10A3A000401C80B2208000EB0801308800F025FBC3
:10A3B0002188084480B22080B28842B1B16871B16E
:10A3C0004044FBF7BFFF2088B188084420806D1C03
:10A3D000EDB297F82C00A842CAD80020D2E7FFE7D8
:10A3E0000720CFE70A78062822F0FF020A7010D271
:10A3F000DFE800F0030507090B0D002008E011203D
:10A4000006E0212004E0312002E0122000E02220BA
:10A4100008707047002805D10349012048700020CA
:10A42000FDF73ABA70470000EC24002010B5162062
:10A43000FCF790FAA0B1114890F8000440090828F0
:10A4400011D20121814011F0EC0F0CD00C48826830
:10A450004FF480016AB1016841F48001016010BDD0
:10A4600042F2010001E042F20200BDE81040FCF7B8
:10A470008DBB4FF0E020C0F8001110BD16E000E0E9
:10A48000D82600202DE9F84F204D924689460646F1
:10A490009846012269461846AF68FDF755F858B34B
:10A4A000009800210446801C09E000BF00EA070371
:10A4B0005AF8212005EB8303401C491CDA60414512
:10A4C000F4D34FEA164AFDF797FB4AEA0041601CB5
:10A4D000384005EB80003C4005EB8402C160D06849
:10A4E00066F3C50068F3891069F39F2020F003002C
:10A4F000401C20F00400D06095F8200402E000BF6A
:10A50000FEF764FC0028FBD1BDE8F88F8828002006
:10A510002DE9F84F1D4C00256846D4E901A6FDF74A
:10A5200075FB002738B30023009A61681CE0D1F85E
:10A5300000C00846944503D9ACEB02020A6015E05E
:10A54000A2EB0C0263440760D0F80CC0C1698146DD
:10A55000BCF1000F08D006EB030828F07F48C0E9E3
:10A56000018CC9F81C5005460029E0D128466160DD
:10A57000FDF7C0FC03E02846FDF7BCFC10B15046D7
:10A58000FDF7ACF9E770BDE8F88F00001823002054
:10A590000D4B10B5596831B102680C68A24204D85D
:10A5A000A21A0A60C161586010BD0B4603E00B4659
:10A5B000C969121B21B10C689442F8D3A41A0C602B
:10A5C0000260C161D86110BD182300202DE9F0415F
:10A5D000144E77683D462C4603E0844204D025465D
:10A5E000E469002CF9D11BE0D4B1A5420BD1F86984
:10A5F000706040B90C49012088600021B160F070A2
:10A600002F20FFF723F92168E069E86110B10268A3
:10A61000114401607068874202D00120BDE8F081DA
:10A620000020FBE718230020001001407CB50646FF
:10A6300000240D468DF800406846FCF743FB01A856
:10A6400000F080FA70B10570094946609DF8040079
:10A6500048709DF80000FCF759FB1420FBF778FFC9
:10A6600020467CBD04249DF80000FCF74FFBF7E773
:10A67000CC2500202DE9F041194D6C68002C2CD020
:10A68000184800270068A968B846401A20F07F469D
:10A690002068B0420CD82146361A0744E469087C89
:10A6A00020B181F81080886949698847002CEFD172
:10A6B00029786878814206D1401CC0B268700228AF
:10A6C00001D185F80180064869780C3040F8217086
:10A6D000BDE8F0411420FBF73BBFBDE8F08100006E
:10A6E000182300200415014070B50C4605464FF4B0
:10A6F0008E71FFF760F8216AA068415C206A401CF7
:10A700002062C5F81C1570BD1FB500228DF8002011
:10A710000291816801914261D0E900126846904738
:10A720001FBD00001FB50A4601788DF80010416872
:10A730000191017A8DF80810C0680390044850F820
:10A740002210001F50F82220684690471FBD0000CD
:10A75000E4220020014901200870704734230020C2
:10A7600010B588B0044620220E496846FBF7EAFD82
:10A7700006200090C01F0190029003904FF0EB70F4
:10A7800006900CB1084A00E0002269460748FEF72F
:10A7900043F808B1FCF7FAF90448001F447008B008
:10A7A00010BD000014AE020055A70200382300209F
:10A7B0002DE9FF470C4605464FF40071FFF701F8FD
:10A7C00001274FF40178002618B34FF492794946D7
:10A7D0002846FEF7EBFFE0B149462846FEF7EBFFBF
:10A7E000C5F8088394F8290000B96F6002208DF83D
:10A7F0000000D5F88004C5F880040390A069029099
:10A80000E0680190A661E661D4E9001268469047CD
:10A8100028E004212846FEF7D4FF18B34FF48471D2
:10A820002846FEF7C3FFE8B121462846FFF7E8FCBB
:10A83000616AA069884215D1E06938B1E268616A4D
:10A84000A0612069E6616662E06008E094F8290092
:10A8500000B96F60C5F80883A661E268616A2046A6
:10A86000FFF7E7FC4FF48E7841462846FEF79EFF3F
:10A8700078B1206A6169884202D294F8280020B336
:10A8800041462846FEF797FF616911B12046FFF760
:10A890003BFF4FF4A27841462846FEF787FF002889
:10A8A00018D041462846FEF786FF94F8290000B1EB
:10A8B0002F60A06900280DD0A661E268616A04B02B
:10A8C0002046BDE8F047FFF7B4BC21462846FFF715
:10A8D0000BFFDEE7BDE8FF871FB50A4601788DF85C
:10A8E000001041680191017A8DF80810C06803904A
:10A8F000044850F82210001F50F822206846904764
:10A900001FBD0000E42200202DE9FF410C464FF45A
:10A91000927706463946FEF75AFF0025B8B1394608
:10A920003046FEF759FF02208DF80000D6F880046B
:10A93000C6F880040390D6F83C050290E0680190C8
:10A94000A561E561D4E900126846904723E04FF421
:10A95000887739463046FEF73AFFE0B1394630464F
:10A96000FEF73AFFD6F83C15A069884213D1E0699A
:10A9700060B1E268D6F8000220F02000C6F80002BC
:10A98000E069A0612069E561E06001E0A561E2683D
:10A990002046FFF759FC4FF4A27739463046FEF7C0
:10A9A00016FF68B139463046FEF716FFA06938B188
:10A9B000A561E561D6F83C152046E268FFF744FC46
:10A9C0004FF4907739463046FEF701FF002812D049
:10A9D00039463046FEF700FF606900280BD0D6F8F4
:10A9E0004C058DF800500290A06801906561D4E993
:10A9F000001268469047BDE8FF810870000A487061
:10AA0000022070472DE9F05F8346DDE90A4A994646
:10AA100090460D460846012703E000BFB0FBF8F062
:10AA20007F1C4045FAD2B94500D94F465FEACA704B
:10AA300012D18CB15FEA8A7002D5B9F1000F01D052
:10AA4000202607E0302605E031465846641EFCF714
:10AA5000C3FD0CB1A742F7D35FF00106B9F1010FB6
:10AA600002D9A9F1010903E0B5FBF6F0404502D394
:10AA700006FB08F6F2E7DFF83C9000BFB5FBF6F006
:10AA800000FB165519F800105846FCF7A5FDB6FB5B
:10AA9000F8F6002EF2D15FEACA7009D0002C07D078
:10AAA000A74205D220215846641EFCF795FDF5E724
:10AAB000BDE8F09F96AC0200F8B5054680B2FDF700
:10AAC00007F9040013D0154E207A0027317B884205
:10AAD0000ED2A8B204F10A0175DF28B1112806D000
:10AAE000BDE8F840FFF712BC207A401C2072F8BD88
:10AAF0002772307C38B1A8B23B2176DF18B1082824
:10AB000001D0FFF703FC71690029F0D08DF80070C7
:10AB1000ADF8025068468847F8BD00005824002070
:10AB200030B40446007A00280AD06088002166DF2D
:10AB300028B1112802D0616830BC0847012020727A
:10AB400030BC70470A494A788B78521CD2B2934283
:10AB500000D100220B78934201D10020704702708F
:10AB6000487800EB400001EBC000001D704700007A
:10AB7000CC2500202DE9FC411646DDE90854CDE93D
:10AB800000541F468046022200F00CF8002807D12E
:10AB9000CDE900543B4610223146404600F002F811
:10ABA000BDE8FC812DE9FC5F0026DDE90C4B9946F0
:10ABB00092468E4680462788354630E0D8F8040015
:10ABC000002200EB850069460068019001A864DF5F
:10ABD000002830D19DF8000050451FD10EB1002152
:10ABE00000E00221228808441118594522D846B9AC
:10ABF000521C90B2208009F800E02088401C208080
:10AC00000126218801A801EB0902694664DF0028BA
:10AC100011D120889DF80010084420806D1CB8F8E0
:10AC20000000A842CADC56B12088C01B401E80B27A
:10AC3000FF2802D90C20BDE8FC9F09F8070000207E
:10AC4000F9E7000023150000111213140D0E0F1068
:10AC5000770A000000000000770A000000000000F2
:10AC60007ADA00000000000023D1BCEA5F782315E7
:10AC7000DEEF12120000000000000050099B0200ED
:10AC8000619D020003000000AC25002000000000D0
:10AC90000338FDD8704730313233343536373839E0
:10ACA000414243444546000000000000000000000F
:10ACB0000000000000000000000000000000000094
:10ACC000A8AC0200C0AC020004000000556E6B6E20
:10ACD0006F776E206572726F7220636F646500001B
:10ACE0000000000088B302000100000034B202003E
:10ACF0000200000028B0020003000000A8B2020019
:10AD000004000000FCB2020005000000DCB10200FB
:10AD10000600000078B1020007000000E4B2020063
:10AD200008000000F0B102000900000054B2020067
:10AD30000A00000070B302000B00000010B0020017
:10AD40000C00000008B202000D000000D8B30200A1
:10AD50000E000000D4B202000F00000010B3020089
:10AD60001000000044B3020011000000ECB3020028
:10AD700012000000C0B30200130000005CB3020028
:10AD80008000000090B1020081000000CCB0020001
:10AD9000820000008CB00200830000006CB0020052
:10ADA00084000000A8B0020085000000B4B10200D9
:10ADB00086000000BCB202009000000058B1020002
:10ADC000910000004CB00200920000001CB2020092
:10ADD0000082000024B302000182000070B2020071
:10ADE000028200008CB2020000840000E8B0020081
:10ADF0000184000094B302000284000030B102001C
:10AE0000038400000CB10200698D02003D8D020038
:10AE1000358D0200FFFFFFFFFFFFFFFFFFFFFFFF7A
:10AE2000FFFFFFFF00000000000000000000D6014F
:10AE300006010000F02700207F000000702800209D
:10AE40000000000000000000000000000000000002
:10AE50000100000740AE020050AE020008000000F2
:10AE600078AE020088AE02000800000088AE020042
:10AE700098AE02000800000058B7020060B7020058
:10AE8000000000000000000048B7020058B70200B0
:10AE9000000000000000000010B7020018B7020018
:10AEA00018B7020028B7020028B7020038B702001E
:10AEB00038B7020040B70200B822002098AE020066
:10AEC000B8AE02000800000040B7020048B7020018
:10AED0000000000000000000C8AE0200D8AE020072
:10AEE0000800000000404040404040404040414198
:10AEF000414141404040404040404040404040404F
:10AF000040404040400502020202020202020202E8
:10AF100002020202022020202020202020202002E5
:10AF20000202020202029090909090901010101075
:10AF30001010101010101010101010101010101011
:10AF400002020202020288888888888808080808A5
:10AF50000808080808080808080808080808080871
:10AF60000202020240000000E5AE020073645F626C
:10AF70006C655F6761705F646174615F6C656E676B
:10AF800074685F7570646174652829202872657122
:10AF90007565737429206F6E20636F6E6E656374C0
:10AFA000696F6E20307825782072657475726E65D1
:10AFB000642025732E000000546865207265717549
:10AFC000657374656420636F6D62696E6174696F27
:10AFD0006E206F6620545820616E64205258207095
:10AFE00061636B6574206C656E6774687320697348
:10AFF00020746F6F206C6F6E67206279202575203A
:10B000006D6963726F7365636F6E64732E00000009
:10B010004E52465F4552524F525F494E56414C493F
:10B02000445F4441544100004E52465F4552524FE6
:10B03000525F534F46544445564943455F4E4F5423
:10B040005F454E41424C4544000000004E52465F71
:10B050004552524F525F464541545552455F4E4FFF
:10B06000545F454E41424C45440000004E52465FFD
:10B070004552524F525F4D555445585F554E4C4FB7
:10B08000434B5F4641494C45440000004E52465FE9
:10B090004552524F525F4D555445585F4C4F434BAC
:10B0A0005F4641494C4544004E52465F4552524F1F
:10B0B000525F4D555445585F434F4E445F494E498A
:10B0C000545F4641494C4544000000004E52465FE3
:10B0D0004552524F525F4D555445585F494E495461
:10B0E0005F4641494C4544004E52465F4552524FDF
:10B0F000525F424C455F495053505F52585F504B2E
:10B10000545F5452554E4341544544004E52465F9D
:10B110004552524F525F424C455F495053505F5029
:10B120004545525F52454A4543544544000000009E
:10B130004E52465F4552524F525F424C455F495016
:10B1400053505F4C494E4B5F444953434F4E4E451D
:10B1500043544544000000004E52465F4552524F52
:10B16000525F4150495F4E4F545F494D504C454DE1
:10B17000454E5445440000004E52465F4552524FE2
:10B18000525F4E4F545F535550504F5254454400F8
:10B190004E52465F4552524F525F4D4F44554C45BB
:10B1A0005F4E4F545F494E495449414C495A4544BA
:10B1B000000000004E52465F4552524F525F4D4FC5
:10B1C00044554C455F414C52454144595F494E49B5
:10B1D0005449414C495A4544000000004E52465FD4
:10B1E0004552524F525F4E4F545F464F554E4400AA
:10B1F0004E52465F4552524F525F494E56414C495E
:10B20000445F5354415445004E52465F4552524F9D
:10B21000525F444154415F53495A45004E52465F84
:10B220004552524F525F494F5F50454E44494E4739
:10B23000000000004E52465F4552524F525F535637
:10B24000435F48414E444C45525F4D495353494E2C
:10B25000470000004E52465F4552524F525F494EE2
:10B2600056414C49445F4C454E475448000000004D
:10B270004E52465F4552524F525F4452565F5457AA
:10B28000495F4552525F414E41434B004E52465F2B
:10B290004552524F525F4452565F5457495F455290
:10B2A000525F444E41434B004E52465F4552524F0F
:10B2B000525F494E5445524E414C00004E52465F3B
:10B2C0004552524F525F53544F524147455F465586
:10B2D0004C4C00004E52465F4552524F525F4E5505
:10B2E0004C4C00004E52465F4552524F525F494E01
:10B2F00056414C49445F504152414D004E52465FC9
:10B300004552524F525F4E4F5F4D454D0000000079
:10B310004E52465F4552524F525F464F5242494449
:10B3200044454E004E52465F4552524F525F445282
:10B33000565F5457495F4552525F4F5645525255DA
:10B340004E0000004E52465F4552524F525F494EEA
:10B3500056414C49445F4144445200004E52465FBE
:10B360004552524F525F5245534F55524345530039
:10B370004E52465F4552524F525F494E56414C49DC
:10B38000445F464C414753004E52465F535543433A
:10B39000455353004E52465F4552524F525F424C06
:10B3A000455F495053505F4348414E4E454C5F41C5
:10B3B0004C52454144595F4558495354530000008D
:10B3C0004E52465F4552524F525F434F4E4E5F437F
:10B3D0004F554E54000000004E52465F4552524FAA
:10B3E000525F54494D454F55540000004E52465F40
:10B3F0004552524F525F4255535900007761726E69
:10B40000696E670064656275670000001B5B313B15
:10B4100033306D001B5B306D000000001B5B313B67
:10B4200033316D001B5B313B33326D001B5B313BB5
:10B4300033336D001B5B313B33346D001B5B313BA1
:10B4400033356D001B5B313B33366D001B5B313B8D
:10B4500033376D00696E666F000000006572726FB1
:10B460007200000073645F626C655F6366675F73A0
:10B47000657428292072657475726E656420257361
:10B48000207768656E20617474656D7074696E678D
:10B4900020746F2073657420424C455F47415454BB
:10B4A000535F4346475F534552564943455F4348C0
:10B4B000414E4745442E000073645F626C655F63D4
:10B4C00066675F73657428292072657475726E658E
:10B4D00064202573207768656E20617474656D70D3
:10B4E00074696E6720746F2073657420424C455FE9
:10B4F000434F4D4D4F4E5F4346475F56535F555543
:10B5000049442E0073645F626C655F6366675F73B6
:10B51000657428292072657475726E6564202573C0
:10B52000207768656E20617474656D7074696E67EC
:10B5300020746F2073657420424C455F474154541A
:10B54000535F4346475F415454525F5441425F53F7
:10B55000495A452E0000000073645F626C655F63AA
:10B5600066675F73657428292072657475726E65ED
:10B5700064202573207768656E20617474656D7032
:10B5800074696E6720746F2073657420424C455F48
:10B59000434F4E4E5F4346475F4741502E000000E9
:10B5A00073645F626C655F6366675F7365742829A7
:10B5B0002072657475726E656420257320776865E6
:10B5C0006E20617474656D7074696E6720746F208D
:10B5D00073657420424C455F4741505F4346475F67
:10B5E000524F4C455F434F554E542E006E72665F6E
:10B5F000626C655F6761747400000000636C6F6368
:10B600006B000000434C4F434B0000004750494F34
:10B610005445000050525300554152540000000060
:10B6200055415254450000007077725F6D676D742C
:10B6300000000000756172745F6C6F675F62616328
:10B640006B656E6400000000617070006E72665F72
:10B65000736468006E72665F7364685F626C650035
:10B660006E72665F7364685F736F630060B7020039
:10B67000B8220020F40000003469020054B802002F
:10B68000AC230020042900004469020008AE020037
:10B690000000000034B602004C230020ECB502008C
:10B6A00000000303FCB502000000000004B6020025
:10B6B000000000000CB602000000000014B60200FA
:10B6C0000000000018B602000000000020B60200D2
:10B6D0000000000028B602000000000048B602008A
:10B6E000000003034CB602000000030354B602003E
:10B6F0000000030360B60200000003035C23002087
:10B70000542300205C230020302700201800000074
:10B71000957202000000000051850200C423002041
:10B7200099710200000000005D740200AC2300204B
:10B73000DB860200D82300209D700200000000007C
:10B7400015A4020000000000D595020000000000D2
:10B75000D59602000000000061A202000000000077
:10B76000FF00FFFF0D0003001D760200E423002010
:10B770001F000000032400201F0000000000000044
:10B7800000000000000000000000000000000000B9
:10B7900000000000000000000000000000000000A9
:10B7A0000000000000000000000000000000000099
:10B7B0000000000000000000000000000000000089
:10B7C0000000000000000000000000000000000079
:10B7D0000000000000000000000000000000000069
:10B7E0000000000000200040000000000020004099
:10B7F0000000000000000000FF000000000000004A
:10B800000000000000000000000000000000000038
:10B8100000000000000000005CB40200FCB3020065
:10B8200054B4020004B4020014B402000CB40200C8
:10B830001CB4020024B402002CB4020034B4020090
:10B840003CB4020044B402004CB40200000000000A
:04B850000090D00391
:040000050002620192
:00000001FF
